:080000002CC0FECFFDCFFCCFA8
:10000800FBCFFACFF9CFF8CFF7CF52C0F5CFF4CF67
:10001800F3CFF2CFF1CFF0CFEFCFEECFEDCF02009D
:1000280002000000000000000000000001002D4E4A
:10003800414E00494E4600000100640126000100BF
:10004800660128000A0004002A0001006801340043
:100058000000F894EE27ECBBF1E0FBBFEBBFE5BF77
:10006800F8E1F1BDE1BD8DE0A2E0BB27ED938A95F3
:10007800E9F780E094E0A0E6ED930197E9F7E0E482
:10008800F0E085919591009761F0A591B591059063
:100098001590BF01F00105900D920197E1F7FB0162
:1000A800F0CFEFE5EDBFE4E0EEBFC0E6D1E0F6C08B
:1000B8000A921A929A93AA93BA93EA93FA93EFB789
:1000C800EA93E5E0E2BFF401309761F4E1E0F0E0A3
:1000D8004F01C29AC198C098D501E4E6F0E017D460
:1000E80005D23EC0E130A0E0FA0721F4E2E0F0E0FA
:1000F8004F012EC0E230A0E0FA0769F4FCD14F01AD
:10010800C298C19AC098D501F9D101D4DF01F6D1BE
:100118003BD4ECD125C0E330A0E0FA0721F4E4E0B9
:10012800F0E04F0115C0E430A0E0FA0759F4E5E02B
:10013800F0E04F01C298C198C09AD501DFD124D40C
:10014800D5D10EC0E530A0E0FA0751F488249924EF
:10015800C298C198C098E0E0E0936001E093610123
:10016800E8ECF0E0AE16BF0610F0CBD108F477C08B
:10017800E0916001F0916101309739F4C7D111F431
:10018800EFEB01C0EFE3E2BB69C0E130A0E0FA07A2
:1001980039F4BCD111F4E6E801C0E6E0E2BB5EC088
:1001A800E230A0E0FA0739F4B1D111F4EBED01C067
:1001B800EBE5E2BB53C0E330A0E0FA0739F4A6D17F
:1001C80011F4EFEC01C0EFE4E2BB48C0E430A0E07A
:1001D800FA0739F49BD111F4E6EE01C0E6E6E2BB7A
:1001E8003DC0E530A0E0FA0739F490D111F4EDEE06
:1001F80001C0EDE6E2BB32C0E630A0E0FA0739F410
:1002080085D111F4EDEF01C0EDE7E2BB27C0E7307F
:10021800A0E0FA0739F47AD111F4E7EA01C0E7E27D
:10022800E2BB1CC0E830A0E0FA0739F46FD111F442
:10023800EFEF01C0EFE7E2BB11C0E930A0E0FA0739
:1002480039F464D111F4EFEE01C0EFE6E2BB06C069
:10025800EA30A0E0FA0711F4E0E0E2BB06C051D1B1
:1002680010F4E6E701C0E8E3E2BB48D1E415F50580
:1002780031F4E1E0F0E03F014424552405C0F201E7
:1002880031962F0166247724E991EFBFF991E9911E
:10029800B991A9919991199009901895E7E0E8BB4F
:1002A800E7BBE0E0E5BBE4BBEFEFE2BBE1BBE3E0CB
:1002B800E3BFE5E0E2BFE1E0E9BFE6E4E7B9E7E88C
:1002C800E6B97894E1E0F0E0E615F70509F097C0A3
:1002D80098D066277727A0EFB8E18CE990E04FD354
:1002E800E051F74260407040C8D1A0E0B5E88FEC1B
:1002F8009AE49BD20FD1A2E6B1E086D1ED93FC93AC
:100308000FD1A5EFBBEC85E799E341D2AFE9B8EC93
:1003180083E99AE3ECD17F936F93FF93EF9300D136
:100328007F936F93FF93EF93FBD0AF91BF918F9122
:100338009F912DD27F936F93FF93EF93F1D0AF915D
:10034800BF918F919F9123D2ABEFB7EB89EB93E3EA
:100358001ED2AF91BF918F919F91C9D1EAD065D23A
:10036800DF01CB01E3E3F3E968E873E428D3B8D10C
:10037800D1D04AD16F01F5013A96CE16DF0628F49E
:10038800F5013A97EC15FD0510F0560132C0AC1492
:10039800BD04B0F4D3D0A0916401B09165011A975F
:1003A80029F4F50131965F01CFD009C0E0916401CD
:1003B800F09165013196E0936401F09365011FC0E7
:1003C800CA14DB04B0F4C0D0A0916601B0916701F3
:1003D8001A9729F4F50131975F01B0D009C0E0916F
:1003E8006601F09167013196E0936601F093670129
:1003F80006C0E0E0E0936401E09365019FD062CF1E
:10040800FFCF369A349BFECF349AE4B1F5B1089504
:100418002497E8D29FD0E0D22CF0EFEFFFEF6FE700
:100428007FEF61C09CD0C6D2EDB7FEB73197FA9383
:10043800EA931F930F93A2D00F911F9195D08AD062
:10044800E3EFF4E065E37FE335D230F488D082D07F
:100458004ED18AD00150104082D06BD041D17F93C9
:100468006F93FF93EF937BD064D041D1AF91BF914D
:100478008F919F91DAD178D072D06CD088D1EA83ED
:10048800FB836C837D8375D0A6E2B2E485E69FE3A7
:100498007ED1DF01CB01EEE4F1E164E570E48FD2B7
:1004A8001FD158D074D17F936F93FF93EF9361D08E
:1004B800ADE4B1E184ED9FE313D1AF91BF918F918A
:1004C8009F91B3D17F936F93FF93EF93F8011AD263
:1004D800D4D0A8E1B2E781E39FE359D1AF91BF91AE
:1004E8008F919F9104D181D22A960895E09360015B
:1004F800F09361010895E3E0F0E00895EAE0F0E0A8
:100508000895E4EFF1E0EA15FB050895F4DFE81536
:10051800F9050895A0E0B0E080E291E438D10895AB
:10052800E0916201F091630166277727A6D042D255
:100538006FCFA0E0B0E080E89FE30895E0E0E093AB
:100548006601E09367010895E0E0E0936401E093B9
:1005580065010895AE81BF81888599850895EE81EA
:10056800FF81688579850895EE83FF836887798799
:100578000895EA81FB816C817D810895A991B991E3
:10058800E991F9916991799177FB660F771F88272F
:100598007E57880B7D938C937EE7769567950EF052
:1005A800089530976040704009F0705808955523B9
:1005B80042F4503811F4E0FF04C03196691F791FE6
:1005C8006BF050E8572711F45F93CFC05F3F31F0CD
:1005D800660F000C57956795752F08955F93002057
:1005E8000AF0CFC0C8C050E8192E1522880F991FED
:1005F8009527550F879550E8072E0522660F771F18
:100608007527550F67950895689401C0E8945F931E
:10061800F2DF703818F07F3F08F4A7C056E1571B87
:10062800AAF4519558300EF4593030F0EFEFFFEF3F
:100638006FEF7FE777F91AC077275523B9F0EE0FE8
:10064800FF1F661F771F5A95D1F710C077275830BC
:1006580028F0EF2FF62F672F5850F9CF552331F098
:1006680076956795F795E7955A95D1F700200AF49E
:1006780041D15F910895689401C0E8943097604033
:100688007040B1F0002426F0772312F4009432D1A0
:10069800172E7EE1112032F07A95EE0FFF1F661FAC
:1006A800111CF9CFEF2FF62F612D5F938ADF5F9131
:1006B80008954F93AF01FD01DA01AB01BC01CA01F6
:1006C800402D012C142E4F910895EA0FFB1F681F2F
:1006D8000895E095F0956095EF5FFF4F6F4F08958F
:1006E8005F9381DF903871F150E8152604C05F935D
:1006F8007ADF903839F1703821F1572F591B2BF1D7
:1007080012F4D7DFFACF583118F0AA27BB27882769
:10071800583028F0AB2FB82F88275850F9CF5523D9
:1007280029F08695B795A7955A95D9F7502D512553
:1007380072F0CBDF38F46795F795E795739513F466
:1007480020C0B7DF3EDF5F910895D8F7FBCFEA1BE3
:10075800FB0B680B51F010F40094BBDF662392F397
:10076800EE0FFF1F661F7A95CBF7EE27FF27662748
:1007780077275F910895EFEFFFEF6FE77FEF5F91C6
:100788000895EFEFFFEF6FE77FE75F9108955F93BD
:100798002ADF703851F3903841F301240894791F07
:1007A80023F41CF300203AF3ECCF0F921F932F93FE
:1007B8003F934F93112722279927689FA0018F9F66
:1007C800302D410D591F6B9F300D411D591F8E9FB4
:1007D80027D0BF9F25D06A9F23D0BE9F1DD0AF9F33
:1007E8001BD0AE9F110D291F391F491F591FE32F19
:1007F800F42F652F522F4F913F912F911F910F90FA
:1008080066232AF0550FEE1FFF1F661F02C073955F
:100818004BF2CDDE5F910895100D211D391F02C0E6
:10082800200D311D491F591F08955F93DCDE703874
:1008380021F411200AF49FCFA4CF903809F495CF62
:1008480001240894970B1BF4D4F30020F3CF792FDD
:100858001F932F933F934F93112411272227332758
:100868004427552790E2AE17BF078607410730F0A7
:10087800AE1BBF0B860B410B089401C08894551F13
:10088800221F331F111CAA1FBB1F881F441F9A95C4
:1008980051F7F901612D4F913F912F911F916623D7
:1008A80032F0550FEE1FFF1F661F7A9543F27FDE69
:1008B8005F91089599239AF0772342F0971748F0AB
:1008C80029F4AE17BF07860720F031F09894889472
:1008D800089598940894089518948894089577230F
:1008E800C2F7971798F3A9F7EA17FB07680788F381
:1008F80099F3ECCFF09560957095E195FF4F6F4FA8
:100908007F4F08956F2F660F660B762F089500248A
:10091800112490E1AA0FBB1F001C111C0E1A1F0AFC
:1009280018F40E0E1F1E01C0A1609A9599F7FD01DB
:10093800D00108953F934F935F93002411244427D7
:10094800552730E2AA0FBB1F881F991F001C111CD6
:10095800441F551F0E1A1F0A460B570B28F40E0E7C
:100968001F1E461F571F01C0A1603A9559F7FD0188
:10097800BC01D001CA015F914F913F91089507D002
:10098800D9DF0EF4B7DF0895C2DFFD010895E894BA
:1009980077FF02C0AFDF689497FF0BC00024A095D3
:1009A800B095809590951196801D901D00F8039440
:1009B80000FA08957A936A93FA93EA930895182EA1
:1009C800862F612D192E972F712D1B2EBF2FF12DDC
:1009D8001A2EAE2FE12D089500240A160B060806DC
:1009E800090608951A930A930895198108810895AC
:00000001FF
